:020000040800F2
:10000000C02D00200502000835120008311200083A
:10001000331200088D050008991700080000000041
:100020000000000000000000000000004501000882
:100030008F05000800000000A1010008BD120008A3
:100040001F0200081F0200081F0200081F0200080C
:100050001F0200081F0200081F0200081F020008FC
:100060001F0200081F0200081F0200081F020008EC
:100070001F0200081F0200081F0200081F020008DC
:100080001F0200081F0200081F0200081F020008CC
:100090001F02000800000000000000001F0200080E
:1000A0001F0200081F0200081F0200081F020008AC
:1000B0001F0200081F0200081F0200081F0200089C
:1000C0001F0200081F0200081F0200081F0200088C
:1000D0001F0200081F0200081F0200081F0200087C
:1000E0001F0200081F020008000000001F02000895
:1000F0001F0200081F0200081F0200081F0200085C
:100100001F0200081F0200081F0200081F0200084B
:100110001F0200081F020008F11200081F02000859
:100120001F0200081F0200081F0200081F0200082B
:10013000DFF80CD000F0B2F8004800476919000859
:10014000C02D00202C4B19680868B0E8F04F80F3F0
:100150000988BFF36F8F4FF0000080F3118870475C
:100160000000000008480068006880F308884FF02D
:10017000000080F3148862B661B6BFF34F8FBFF3FF
:100180006F8F00DF00BF00BF08ED00E0DFF80C005C
:10019000016841F470010160704700BF88ED00E024
:1001A000EFF30980BFF36F8F134B1A681EF0100F27
:1001B00008BF20ED108A20E9F04F106009B44FF01D
:1001C000500080F31188BFF34F8FBFF36F8F02F0A1
:1001D0002FF84FF0000080F3118809BC19680868F7
:1001E000B0E8F04F1EF0100F08BFB0EC108A80F39B
:1001F0000988BFF36F8F70471C000020EFF3058064
:10020000704700000648804706480047FEE7FEE7C3
:10021000FEE7FEE7FEE7FEE7FEE7FEE7FEE7FEE7B6
:10022000D11200083101000840EA01039B0703D006
:1002300009E008C9121F08C0042AFAD203E011F825
:10024000013B00F8013B521EF9D27047D2B201E0E7
:1002500000F8012B491EFBD270470022F6E710B5CB
:1002600013460A4604461946FFF7F0FF204610BD24
:1002700030B50B46014600202022012409E021FA76
:1002800002F59D4205D303FA02F5491B04FA02F573
:100290002844151EA2F10102F1DC30BD064C074DC9
:1002A00006E0E06840F0010394E807009847103446
:1002B000AC42F6D3FFF740FFF42C0008142D0008E1
:1002C000FEE700F0DFBA00002DE9F041C2B048229D
:1002D000654930A8FFF7A8FF48211EA8FFF7BDFF1A
:1002E00028226149483114A8FFF79EFF28225E4961
:1002F00070310AA8FFF798FF28216846FFF7ADFF85
:1003000000245B4D5948A8605A48A8605A48E860E4
:100310005A48E8605A48C5F88C025A48C5F88C0219
:1003200030AE1EAF032156F824201068C3439BB2A1
:10033000B3EB104F02D147F8240001E0491EF4D17D
:1003400009B9FFF7BEFF641C122CEBD31E981F994E
:10035000C0F30B00C1F30B0140EA0140009020986C
:10036000C0B201902198229900F00F0001F01F0106
:1003700040EA0140029023982499C0F30A00C1F397
:100380000C0140EA0140039025982699C0F30A0029
:10039000C1F30A0140EA014004902798289900F02F
:1003A0003F0001F03F0140EA01400590299800F02C
:1003B0003F000690DDE92A0161F31F400790DDE967
:1003C0002C0161F31F4008902E982F99C0F30B0069
:1003D000C1F30B0140EA01400990002014AE0DF179
:1003E00028086F4656F820100C6858F8202057F857
:1003F00020301440A34203D00C6894431C430C608B
:10040000401C0A28EED3D5F8000240F00100C5F8E0
:10041000000200BF00BF00BF00BF00BF00BF00BFA1
:1004200000BF00BF00BFD5F8000220F00100C5F8F2
:100430000002002456F82400006858F8241057F8E9
:10044000242001408A4201D0FFF73BFF641C0A2CA4
:10045000F0D3686940F080406861686940F000400E
:10046000686142B0BDE8F081542C00082301674563
:1004700000200240AB89EFCD3B2A19087F6E5D4C0E
:1004800051407F5D6327CE4610B590B02C2105A862
:10049000FFF7E3FE14216846FFF7DFFE1F200590FB
:1004A000002406940B9401200A9008940C940D905B
:1004B00005A800F043FB08B1FFF702FF0F200090F2
:1004C0000194029403944FF48060049000216846E4
:1004D00000F0EAF9002801D0FFF7F2FE10B010BDDD
:1004E00030B587B0142102A8FFF7B7FE0021244CD5
:1004F000E06940F40030E061E06900F40030019010
:100500002148204A02604FF4E13242608160C160BC
:10051000016181610C224261C161016200F0E7FD6D
:10052000606B40F004006063606B00F004000190B9
:10053000606B40F004006063606B00F004000190A9
:1005400004200290022403940120049003200590CB
:1005500006944FF0904502A9284600F019F80821AA
:100560000291069402A9284600F012F80122002107
:10057000262000F055F9262000F044F907B030BDE0
:100580000010024000440040C0000020FEE7704719
:100590002DE9F84F0022DFF87081DFF86CA14FF0F1
:1005A000010E4FF00F0C08F104090AF10C0AA4E047
:1005B0000EFA02F63340002B70D04C68022C01D0AA
:1005C000122C11D1D40800EB84073D6A5407E40EC5
:1005D0000CFA04FB25EA0B05D1F810B00BFA04FB6A
:1005E0004BEA050BC7F820B0076854000325A54067
:1005F000AF4391F804B00BF0030B0BFA04FB4BEA8A
:10060000070BC0F800B04F68012F05D0022F03D0B0
:10061000112F01D0122F11D18768AF43D1F80CB040
:100620000BFA04FB4BEA070BC0F808B04768B74366
:100630000E79C6F3001696403E434660C668AE4348
:100640008D68A5403543C5604C68E40054D52F4CF7
:10065000A56945F00105A561A46904F001040094B1
:100660002B4C22F003052E1977699407250F0CFAFD
:1006700005F4A743B0F1904F04D0264CA04203D11B
:10068000012412E0002410E0234CA04201D10224F6
:100690000BE0224CA04202D1032406E02CE0204CC7
:1006A000A04201D1042400E00724AC403C43746123
:1006B000D8F800409C434D68ED0300D51C43C8F8B2
:1006C0000040D9F800409C434D68AD0300D51C4361
:1006D000C9F800400C4D08352C689C434E68F60262
:1006E00000D51C432C60DAF800409C434D68AD02F5
:1006F00000D51C43CAF80040521C0B6833FA02F4C0
:100700007FF456AFBDE8F88F0004014000100240AE
:10071000000001400004004800080048000C0048A8
:100720000010004801488068704700001000002059
:1007300002488168027811448160704710000020EF
:1007400010B5042000F08CF8072000F005F800F048
:1007500043F8002010BD000000B587B0014600221C
:10076000362000F05DF8362000F04CF81648C169DC
:1007700041F01001C161C06900F01000009001A9B2
:1007800002A800F03BF90598B8B100F05BF9400011
:100790000E49B0FBF1F1491E0E480D4A026040F2CD
:1007A000E732C2604160002101618160816100F037
:1007B000B3FB28B1012007B000BD00F043F9E7E723
:1007C000044800F0C6FBF6E70010024040420F006C
:1007D000001000408000002008B50948816941F000
:1007E00001018161816901F001010091C16941F05C
:1007F0008051C161C06900F08050009008BD0000C8
:1008000000100240002809DB00F01F020121914086
:100810004009800000F1E020C0F80011704700009E
:10082000F0B40D460D4B1B68C3F30223C3F107045C
:10083000032C00D90324D91C072901D2002300E08E
:100840001B1F012606FA04F1491E294099409E40CB
:10085000761E16403143F0BC00F0B0BF0CED00E056
:1008600000F00701054A10684FF6FF03184040EA00
:100870000120034908431060704700000CED00E0C0
:100880000000FA05BFF34F8F05480168054A01F4DF
:10089000E06111430160BFF34F8F00BFFDE700002F
:1008A0000CED00E00400FA052DE9F04704460D4682
:1008B000002C17D0DFF83081D8F8000000F00F00CE
:1008C000A84211D2D8F8000020F00F002843C8F841
:1008D0000000D8F8000000F00F00A84204D001206A
:1008E000BDE8F0870120FBE72068404E810712D564
:1008F000400703D5706840F4E0607060207800071E
:1009000003D5706840F4605070607068A16820F092
:10091000F000084370602078C0072CD06068012880
:1009200006D0022809D0316889070BD40120D7E707
:100930003168890306D40120D2E73168C90101D4A6
:100940000120CDE7716821F0030101437160FFF7D9
:10095000E9FE074641F2883906E0FFF7E3FEC01BD7
:10096000484501D90320BBE77068616800F00C00BE
:10097000B0EB810FF1D1D8F8000000F00F00A842D1
:100980000ED9D8F8000020F00F002843C8F8000066
:10099000D8F8000000F00F00A84201D001209FE726
:1009A0002078400705D57068E16820F4E0600843CE
:1009B00070602078000706D57068216920F46050C7
:1009C00040EAC100706000F05DF87168084AC1F348
:1009D0000311515CC8400749086007480068FFF7E9
:1009E000BBFE00207CE70000002002400010024017
:1009F000442C000800000020140000200F22026098
:100A00000B4A536803F003034360536803F0F00399
:100A10008360536803F4E063C360526802F4605279
:100A2000D20802610348006800F00F0008607047B8
:100A3000001002400020024001480068704700009A
:100A40000000002000B5FFF7F7FF04494968044A99
:100A5000C1F30221515CC84000BD000000100240FB
:100A6000EC2C000800B5FFF7E7FF04494968044A89
:100A7000C1F3C221515CC84000BD0000001002401B
:100A8000EC2C000800B591B0402218A101A8FFF796
:100A9000CBFB26A000680090254A516801F00C00AD
:100AA000042804D0082804D0224811B000BD2248F0
:100AB000FBE701F4701001F0C04340EAD31001AB32
:100AC00003EB90400078C1F30141012904D00329D0
:100AD00002D018494843E8E75168C1F340411DF886
:100AE0000110154A5043B0FBF1F0DEE702030405A4
:100AF000060708090A0B0C0D0E0F1011121314151E
:100B0000161718191A1B1C1D1E1F2021222324250D
:100B1000262728292A2B2C2D2E2F303132333435FD
:100B2000363738393A3B3C3D3E3F3F3F01020000FB
:100B30000010024000127A0000366E012DE9F843E1
:100B40000446002C0ED02078EE4DC00768D06868AF
:100B5000C0F3810001281FD06868C0F3810002281B
:100B600003D006E00120BDE8F8836868C00313D411
:100B7000686860684FF48032904205D1A86BA16824
:100B800020F440700843A863606890420BD1286845
:100B900040F48030286012E02868800340D5606807
:100BA00078BB0120DFE780B1B0F5A02F16D0286810
:100BB00020F480302860286820F480202860606855
:100BC00000B3FFF7AFFD064618E0286820F4803038
:100BD0002860286820F480202860F0E7286840F426
:100BE00080202860286840F480302860E7E7FFF71D
:100BF00099FD801B642801D90320B4E7286880038D
:100C0000F5D50DE0FFF78EFD064606E0FFF78AFDFD
:100C1000801B642801D90320A5E728688003F5D448
:100C2000207880073BD5686810F00C0F08D0686802
:100C3000C0F3810002280BD16868C00308D468683B
:100C4000286880072BD56069012828D001208AE711
:100C5000606990B1286840F001002860FFF762FDEC
:100C6000064606E0FFF75EFD801B022801D903203F
:100C700079E728688007F5D511E0286820F00100A1
:100C80002860FFF74FFD064606E0FFF74BFD801B8F
:100C9000022801D9032066E728688007F5D4207868
:100CA000C00626D5A06990B1A86A40F01000A862DD
:100CB000FFF738FD064606E0FFF734FD801B0228EB
:100CC00001D903204FE7A86A8006F5D511E0A86A8C
:100CD00020F01000A862FFF725FD064606E0FFF7AA
:100CE00021FD801B022801D903203CE7A86A800669
:100CF000F5D42078000729D5E069A8B1686A40F0EA
:100D000001006862FFF70EFD064606E0FFF70AFDE8
:100D1000801B022801D9032025E7686A8007F5D5E2
:100D2000012000F0B9FA11E0686A20F00100686261
:100D3000FFF7F8FC064606E0FFF7F4FC801B0228EC
:100D400001D903200FE7686A8007F5D420784007AF
:100D50007BD54FF00008E869C00009D4E86940F08D
:100D60008050E861E86900F0805000904FF0010881
:100D7000654E3068C00511D4306840F48070306032
:100D8000FFF7D0FC074606E0FFF7CCFCC01B642849
:100D900001D90320E7E63068C005F5D5E0680128F1
:100DA00005D1286A216920F0180008432862E0680C
:100DB000012812D0B0B105281DD0286A20F001000A
:100DC0002862286A20F004002862E06841F2883630
:100DD00028B3FFF7A7FC07461DE0286A40F0010092
:100DE0002862F2E7286A20F001002862286A20F0D1
:100DF00004002862E9E7286A40F004002862286AB3
:100E000040F001002862E0E7FFF78CFCC01BB04215
:100E100001D90320A7E6286A8007F5D50EE0FFF781
:100E200081FC074607E0FFF77DFCC01BB04202D9FA
:100E3000032098E609E0286A8007F4D4B8F1010F8E
:100E400003D1E86920F08050E861206A80B36968C6
:100E5000C1F38101022942D0022807D0286820F07E
:100E600080702860FFF75EFC044634E0286820F0BC
:100E700080702860FFF756FC064606E0FFF752FC3C
:100E8000801B022801D903206DE628688001F5D473
:100E9000D4E90901084369681C4A114008436860A5
:100EA000286840F080702860FFF73CFC044607E0AB
:100EB00026E0FFF737FC001B022801D9032052E689
:100EC00028688001F5D51BE0FFF72CFC001B0228E9
:100ED00001D9032047E628688001F5D410E00128F5
:100EE0000CD06868626A00F48031914204D10849EC
:100EF0000840A16A884203D0012034E6012032E68E
:100F0000002030E60010024000700040FFFFC09F4C
:100F100000003C607047704710B50446002C03D0B9
:100F200094F83D0010B107E0012010BD002084F8C6
:100F30003C00204600F00CF8022084F83D00211D02
:100F4000206800F0DBF9012084F83D00002010BD8E
:100F500070470168CA6842F00102CA60006881688F
:100F600001F00701062903D0016841F00101016089
:100F700000207047704770B50446206801694FF043
:100F80000005C943890716D4C168C943890712D42B
:100F9000E91E01610120207720688069800703D065
:100FA0002046FFF7E7FF05E0204600F09BF82046CB
:100FB00000F099F8257720680169C943490718D4DA
:100FC000C168C943490714D46FF0040101610220CC
:100FD00020772068806910F4407F03D02046FFF717
:100FE000C9FF05E0204600F07DF8204600F07BF8C0
:100FF000257720680169C943090717D4C168C94327
:10100000090713D46FF008010161042020772068DC
:10101000C069800703D02046FFF7ACFF05E02046FB
:1010200000F060F8204600F05EF82577206801693E
:10103000C943C90618D4C168C943C90614D46FF09E
:1010400010010161082020772068C06910F4407FFA
:1010500003D02046FFF78EFF05E0204600F042F85F
:10106000204600F040F8257720680169C943C90788
:1010700008D1C168C943C90704D1891E016120464E
:1010800000F032F820680169C943090609D4C16833
:10109000C943090605D46FF0800101612046FFF7BE
:1010A00039FF20680169C943490609D4C168C943A9
:1010B000490605D46FF040010161204600F016F8A2
:1010C00020680169C94389060BD4C168C9438906F0
:1010D00007D46FF0200101612046BDE87040FFF7A2
:1010E0001ABF70BD70477047FFF722BB704770B5DD
:1010F0000446002C04D094F84500002510B106E009
:10110000012070BD84F84450204600F027F82420C8
:1011100084F845002068C16821F40051C160204670
:1011200000F004FA206A10B1204600F0E7F92068C8
:10113000016921F4904101612068416921F02A018F
:1011400041612068C16841F40051C160A56420205C
:1011500084F8450084F84600002070BD70472DE9F2
:10116000F84F04460E4615461F4694F845002028C1
:1011700002D00220BDE8F88F46B13DB1A0684FF41F
:10118000805A504508D1206910B105E00120F1E7EF
:10119000F00701D00120EDE794F84400012816D0B3
:1011A000012084F844004FF00008C4F84880212052
:1011B00084F84500FFF7B6FA814625866586A06863
:1011C000504501D1206920B13546002615E00220A6
:1011D000D0E7002511E04B460022802120460097F1
:1011E00000F0A8FA08B10320C4E79DB1216815F802
:1011F000010B4860608E401E6086608E0028EAD138
:101200004B46002240212046009700F093FA40B15F
:101210000320AFE736F8020B2168C0F308004860EE
:10122000E8E7202084F8450084F844800020A1E706
:10123000FEE7FEE77047000010B5022001F065F8F8
:101240000D4CA06010B10DA000F0A8FA0121002201
:10125000084601F05EF8206003220021012001F021
:1012600058F86060A168206801F03CF8D4E90101F9
:10127000BDE8104001F036B80400002071756575B6
:10128000652073657420637265617465207375638E
:1012900063657373210D0A0008B507494FF4FA52CC
:1012A0000968B1FBF2F14143009100BF0098411E73
:1012B0000091FAD208BD00000000002010B501F036
:1012C00097FA012803D0BDE8104000F0F5BF10BD2B
:1012D00010B5FEF7F9FF0548016841F4700101609F
:1012E00002494FF000608039086010BD88ED00E0D1
:1012F0000148FFF740BE0000800000202DE9F041CA
:101300000268264D264E274FDFF89CC0274B4FF032
:101310008048A84209D0404507D0B04205D0B84225
:1013200003D0604501D0984203D122F070044A688E
:101330002243A8421BD0404519D0B04217D0B84232
:1013400015D0604513D0984211D0194CA0420ED050
:10135000184CA0420BD0184CA04208D0174CA04209
:1013600005D0174CA04202D0164CA04203D122F463
:101370004074CA6822434C6922F080022243026012
:101380008A68C2620A688262A84201D0984201D18A
:101390000969016301214161BDE8F081002C014030
:1013A0000004004000080040000C004000340140F0
:1013B000004C014000500140005401400018004022
:1013C000001C00400020004008B500250095144C8A
:1013D0009DF800000A2809D100235A1E694620689A
:1013E00001F002F810B10FA000F0D8F99DF800004C
:1013F000142809D100231A461946606800F0F4FF4A
:1014000010B110A000F0CAF99DF80000401CC0B255
:101410000090152800D10095642000F053FED7E716
:10142000040000205461736B313A20717565756555
:101430002073656E642073756363657373210D0A91
:10144000000000005461736B313A2073656D617068
:10145000686F72652072656C656173652073756372
:1014600063657373210D0A0008B500200090104CCD
:10147000451E2946A06801F0BFF8216888420BD1BB
:101480002A46694601F040F80128F2D19DF8001083
:1014900008A000F083F9ECE761688842E9D12946A9
:1014A00001F0B4F80128E4D10BA000F077F9E0E7EF
:1014B000040000205461736B323A20526563656901
:1014C00076652071756575652076616C7565203D62
:1014D0002025640D0A0000005461736B323A2054D9
:1014E000616B652073656D6170686F7265207375DF
:1014F0006363757373210D0A0000000090F82010DB
:10150000490611D501684A69436A22F480521A4398
:101510004A61416AB1F5805F06D101684A69806A13
:1015200022F4C04202434A61704700002DE9F041B5
:10153000044620680169E26821F4405111430161C9
:10154000A16820690143606901432068C26841F2D3
:101550000C639A430A43C26020684169A26921F47E
:1015600040711143416120684169E26921F40061E1
:1015700011434161E1696E4864253226B1F5006F7F
:1015800035D0216881427CD1FFF76CFA00EBC001B5
:1015900001EB001061686FF018078900B0FBF1F2F1
:1015A000B2FBF5F2B0FBF1F37A4303EB8202B0FB3E
:1015B000F1F306EB0212B2FBF5F2B3FBF5F302F026
:1015C000F00202EB0312B0FBF1F3B0FBF1F0B0FB61
:1015D000F5F0784303EB800006EB0010B0FBF5F06C
:1015E000216800F00F0010448860BDE8F081216898
:1015F000814234D1FFF736FA00EBC00101EB001055
:1016000061686FF0180C4900B0FBF1F2B2FBF5F223
:101610001301B0FBF1F2B2FBF5F2B0FBF1F702FB04
:101620000CF207EB820206EBC202B2FBF5F202F00B
:10163000F80203EB4202B0FBF1F3B0FBF1F0B0FBB8
:10164000F5F000FB0CF003EB800006EBC000B0FBF4
:10165000F5F0216800F0070010448860C5E7FFF747
:10166000F1F900EBC00101EB001061684900B0FB2B
:10167000F1F2B2FBF5F21301B0FBF1F7B0FBF1F2BE
:1016800000E023E0B2FBF5F26FF0180C02FB0CF265
:1016900007EB820206EBC202B2FBF5F202F0F8029F
:1016A00003EB4202B0FBF1F3B0FBF1F0B0FBF5F05D
:1016B00000FB0CF003EB800006EBC000B0FBF5F084
:1016C000216800F00700104488608EE7FFF7BAF940
:1016D00000EBC00101EB001061686FF01807890092
:1016E000B0FBF1F2B2FBF5F2B0FBF1F37A4303EB9E
:1016F0008202B0FBF1F306EB0212B2FBF5F2B3FB90
:10170000F5F302F0F00202EB0312B0FBF1F3B0FBD1
:10171000F1F0B0FBF5F0784303EB800006EB00102E
:10172000B0FBF5F0216800F00F00104488605CE722
:10173000003801402DE9F04104460E461746984610
:10174000069D1DE0681C1BD02DB1FEF7EBFFA0EB42
:101750000800A84214D92068C16821F4D071C16082
:101760002068416921F001014161202084F8450091
:1017700084F84600002084F844000320BDE8F0818E
:101780002068006836EA000004D00020B842D9D0B2
:101790000020F3E70120F9E7FEE700000FB4054B56
:1017A00010B503A9044A029800F028F810BC5DF8AF
:1017B00014FB0000511900087C0000204907090EA5
:1017C000002804DB00F1E02080F80014704700F0EE
:1017D0000F0000F1E02080F8141D704702E008C8F7
:1017E000121F08C1002AFAD170477047002001E09B
:1017F00001C1121F002AFBD1704700002DE9FF4FE5
:1018000089B09B460446002506E025280BD05A46A1
:101810000B999047641C6D1C20780028F5D10DB001
:101820002846BDE8F08F0027B8460122474900E06E
:10183000074314F8013F203B02FA03F00842F7D1B6
:1018400020782E2819D114F8010F47F004072A2810
:101850000ED06FF02F022078A0F1300109290CD8AA
:1018600008EB880102EB410100EB0108641CF2E780
:101870000A98641C50F8048B0A9020780028CED077
:10188000642808D0692806D075281ED05A460B99BE
:1018900090476D1C58E00A994FF00A0901C90A9156
:1018A000002802DA40422D2102E0390504D52B211F
:1018B0008DF82010012103E0F90704D02021F7E77B
:1018C0008A4608AE0DE00021FAE70A994FF00A09AE
:1018D00001C90A91F7E74946FEF7CAFC303106F81C
:1018E000011D0028F7D1ADEB060000F120097807B3
:1018F00001D44FF00108C84502DDA8EB090000E063
:1019000000208046002706E008A85A46C05D0B99D3
:1019100090476D1C7F1C5745F6DB04E030205A468B
:101920000B9990476D1CB8F10001A8F10108F5DC96
:1019300005E016F8010B5A460B9990476D1CB9F15A
:101940000001A9F10109F4DC641C65E70928010024
:1019500013B54FF47A73012269460248FFF7FFFB83
:1019600000981CBDC00000201CB5FEF7E9FEFEF784
:101970008BFDFEF7B5FD00240120CDE900042346D0
:10198000802209A10A4800F0FFFE0220CDE90004F0
:101990000023802207A1094800F0F6FEFFF74CFC67
:1019A00000F016FC00201CBD5461736B3100000078
:1019B000C91300085461736B3200000069140008F9
:1019C0002DE9F04104460F461E4DEE682868001DC3
:1019D00000F0EAFA38B9286890F82C100120884005
:1019E000296981432961601C15D1A7B1164948684E
:1019F0002A68906082682B68DA602A688368121D02
:101A00005A602A68121D8260286841610868401C7B
:101A10000860BDE8F081344428684460B44206D2CE
:101A20002968E86B091DBDE8F04100F0E5BA2968B6
:101A3000A86B091D00F0E0FAA86A8442E9D2AC6202
:101A4000E7E700001C000020AC01002070B5044650
:101A500000F0EAFA244DA868401CA860286810B17C
:101A6000686938B10CE02C60A868012808D100F042
:101A70003FF905E02868E16AC06A884200D82C6016
:101A8000686A401C6862E06A01212A69814011434A
:101A90002961164A00EB800002EB80004068A060DC
:101AA0008168E1608368211D59608160E06A00EB14
:101AB000800002EB8001616152F82010491C42F85D
:101AC000201000F0BFFA686900280CD02868E16A8D
:101AD000C06A884207D206494FF080500860BFF3C1
:101AE0004F8FBFF36F8F70BD1C0000200C010020D2
:101AF00004ED00E070B50C4D0C4E11E000F094FACE
:101B0000F068C468201D00F04FFAA868401EA86065
:101B10006868401E686000F095FA204600F053F8AF
:101B200068680028EAD170BD1C00002098010020E0
:101B300030B40B46026C002A0CD0C1681144C1605D
:101B40008468A14201D30168C160C16830BC1846F5
:101B5000FEF76ABB30BC70472DE9F04104461746DA
:101B60000026A56B226C002A10D0C7B1E068FEF7F2
:101B70005BFBE168206C091AE1602268914202D2A5
:101B8000A168081AE060022F16D017E02068A8B9F3
:101B9000A06800F0C9FE06460020A0600EE0606864
:101BA000FEF742FB216C606808446060A1688842CF
:101BB00004D32068606001E005B16D1E6D1CA56353
:101BC0003046BDE8F08110B50446206B00F046FABF
:101BD0002046BDE8104000F041BA416A002904D017
:101BE000006B0068C0F104007047002070470000DF
:101BF0004FF420510E48420706D0C01D20F00700C8
:101C00000B49411AC1F520510A4B186000225A6055
:101C10000144083921F00701143B19604A600A6049
:101C20000A1A42600160406898605860704700007E
:101C3000C001002070000020074E4FF08054074D77
:101C4000FFF758FF30680128FAD92C60BFF34F8F97
:101C5000BFF36F8FF4E700000C01002004ED00E0FB
:101C600010B5029C002909D02260E06321640121A3
:101C7000204600F06FFB0020A06410BD2460F4E754
:101C80002DE9F0478146DDE908560A9C9846521E28
:101C9000206B00EB820020F0070700290CD0002009
:101CA00023180A5C83F834200A5C12B1401C102807
:101CB000F6D3002084F84300042D00D30325E56209
:101CC0006564201D00F095F904F1180000F091F909
:101CD0002461C5F10400A061646242464946384669
:101CE00000F050F92060002E00D03460BDE8F0878D
:101CF00070B50024124D04EB840005EB800000F069
:101D00006DF9641C042CF6D30D48503000F066F9D0
:101D10000B48643000F062F90948783000F05EF951
:101D200007488C3000F05AF90548A03000F056F909
:101D300003490448503181631431C16370BD000010
:101D40000C0100201C00002030B5134900E01146B2
:101D50000A688242FBD34B685C18844203D1406816
:101D60001844486008460D6844682318AB420DD1FA
:101D7000094B143B1B689A4206D0526822444260C9
:101D80000A681268026002E0036000E002608142BB
:101D900000D0086030BD00007000002010B504467F
:101DA00000F042F9A06B20B1002400F04BF920466E
:101DB00010BD0124F9E710B5044600F035F9A06B19
:101DC000E16B884201D1012400E0002400F03AF9DF
:101DD000204610BDF1B50098846C0026A06BE16B25
:101DE000884210D294F94550002269462046FFF7F8
:101DF000B3FE0646681C08D000F0EAF8854202D21D
:101E00006D1C84F845503046F8BD606A0028FAD051
:101E100004F1240000F028FE0028F4D00126F2E7A7
:101E20000648816B0968002904D0816BC96809687C
:101E3000816270474FF0FF31816270471C000020C3
:101E4000502080F31188BFF34F8FBFF36F8FFEE7F1
:101E50002DE9F041044600F0E7F894F9455004F10B
:101E6000240612E0A06C30B12046FFF7B3FF50B15A
:101E700000F04AF907E0606A48B1304600F0F4FD2E
:101E800008B100F041F96D1E6DB2002DEADC4FF093
:101E9000FF3684F8456000F0D5F800F0C5F894F9F5
:101EA000445004F1100709E0206948B1384600F0B9
:101EB000DBFD08B100F028F96D1E6DB2002DF3DCDA
:101EC00084F84460BDE8F04100F0BCB82DE9F04171
:101ED0000546002600F0A4F9234F386808B9FFF73B
:101EE00087FE4DB105F00700C0F11000C1438D42DF
:101EF00001D8054400E00025002D2FDD78688542DB
:101F00002CD8194914310846046801E021460446DA
:101F10006068A84202D220680028F7D1386884425D
:101F20001CD00E680836206808606068411B1029C4
:101F300004D9601941606560FFF706FF6168786841
:101F4000401A7860BA68904200D2B86041F0004010
:101F5000606000202060F868401CF86000F0E8FD38
:101F60003046BDE8F08100005C00002004490868AC
:101F7000002803D00868826C521C8264086870478D
:101F80001C00002024384FF08073036221F001010F
:101F9000C1610449816142606FF0020140F820197B
:101FA00070470000411E00080169D0E901329A60C3
:101FB000D0E901235A604A68824201D182684A60AE
:101FC000002202610868401E08600868704700002F
:101FD00001488068704700001C00002000F10801E3
:101FE00041604FF0FF328260C160016100210160F9
:101FF000704700210161704730B50C68621C02D047
:1020000000F1080202E0026904E01A4653681D6804
:10201000A542FAD953684B6099608A6051600861A3
:102020000168491C016030BD502080F31188BFF366
:102030004F8FBFF36F8F02480168491C01607047E2
:102040007800002004490868401E0860002801D17B
:1020500080F31188704700007800002070B50028D8
:102060001BD0083804466068002816DA2168002969
:1020700013D120F00040606000F0D2F8074D606896
:102080006968084468602046FFF75EFE2869401CC6
:102090002861BDE8704000F04BBD70BD5C000020C1
:1020A0004FF0E02000210161816105494FF47A720F
:1020B0000968B1FBF2F1491E4161072101617047D6
:1020C0000000002010B502460020002A07D000F0D2
:1020D000A7F800211046FFF773FC00F029FD002847
:1020E00007D104494FF080500860BFF34F8FBFF312
:1020F0006F8F10BD04ED00E002490A6A0260C968F2
:10210000416070471C00002001490120C8617047F0
:102110001C00002010B50C46054909681831FFF76E
:102120006BFF2046BDE810400121FFF749BC0000CD
:102130001C00002070B50446002844D0606C884222
:1021400000D30146E06A88423DD0A26C012A3AD110
:10215000E162A269002A02DBC1F10401A1611A4D0A
:1021600000EB8000616905EB800081422BD1201DCE
:10217000FFF71AFF1549012230B994F82C000B69BA
:1021800002FA00F083430B61E06A0B6982401A4354
:102190000A6100EB800005EB80004068A060816868
:1021A000E1608268211D51608160E06A00EB80007F
:1021B00005EB80006061E06A00EB800055F82010BC
:1021C000491C45F8201070BD0C0100201C000020A7
:1021D0007CB50F480025CDE900502B4680220DA18B
:1021E0000E4800F0D1FA0A4C2C3C01280ED15020A8
:1021F00080F31188BFF34F8FBFF36F8F4FF0FF3025
:10220000A06201206061E56000F036F8206B7CBDC3
:102210004800002049444C4500000000391C0008DB
:102220000248416B491C4163704700001C000020BC
:102230000F4A506B002802D00120D0617047002067
:10224000D0611069B0FA80F0C0F11F00094900EBBD
:10225000800001EB800041684968416000F108039B
:10226000994201D1496841604068C0681060704778
:102270001C0000200C01002010B50C48016841F43E
:1022800070010160016841F070410160FFF708FFD3
:10229000074900200860FDF779FF0648016841F012
:1022A00040410160FDF75EFF002010BD20ED00E021
:1022B0007800002034EF00E010B5502080F3118842
:1022C000BFF34F8FBFF36F8F00F0A0FA18B104492E
:1022D0004FF080500860002080F3118810BD00008E
:1022E00004ED00E070B504460D46FFF79DFEA06CBE
:1022F00008B1002405E0A06B08B1002401E0A5644A
:102300000124FFF79FFE204670BD00220421AFF399
:102310000080F8B505460E4617460024002D16D05D
:10232000601EB0FBF5F0B04211D305FB06F010F1D2
:102330004D0F0CD84C30FFF7C9FD04463CB1224686
:102340004C323B46314628460094FFF789FC204634
:10235000F8BD00002DE9F04104460F460125002C90
:102360003BD0E26BC2B3AE1EB6FBF2F1206C8142F1
:1023700033D3FFF759FED4E90F20216802FB001187
:10238000A1600021A16321686160E06B2268216C7B
:10239000401E00FB0121E16084F8446084F8456040
:1023A00004F1100047B1FFF719FE04F12400FFF714
:1023B00015FEFFF747FE11E021690029F9D000F072
:1023C00053FB0028F5D007494FF080500860BFF359
:1023D0004F8FBFF36F8FECE7FFE700252846BDE87E
:1023E000F081000004ED00E02DE9FF4782B00446D3
:1023F0008A4698460025A9464FF08056414FFFF780
:1024000013FEA06BE16B884206D3B8F1020F03D034
:10241000049880B385B338E0A56B42465146204608
:10242000FFF79AFBA16C69B1B8F1020F00D1E5B9D1
:102430002046FFF7CFFCC0B13E60BFF34F8FBFF324
:102440006F8F12E0616A51B104F1240000F00CFBBF
:1024500058B13E60BFF34F8FBFF36F8F05E020B1DF
:102460003E60BFF34F8FBFF36F8FFFF7EBFD01208F
:1024700006B0BDE8F08700E003E0FFF7E3FD0020D1
:10248000F6E76846FFF738FE0125FFF7DBFDFFF7AB
:10249000C7FEFFF7C9FD94F94400401C01D184F840
:1024A000449094F94500401C01D184F84590FFF711
:1024B000C9FD04A9684600F03BF930B12046FFF79A
:1024C000C7FC00F035FB0020D2E72046FFF773FC85
:1024D00088B104F110000499FFF71CFE2046FFF7B5
:1024E000B7FC00F025FB002889D13E60BFF34F8F79
:1024F000BFF36F8F83E72046FFF7AAFC00F018FBBD
:102500007DE7000004ED00E02DE9F74783B00446C5
:102510008A46002600274FF08058DFF8D890FFF752
:1025200083FDA56BC5B151462046FFF701FB6D1E2B
:10253000A563206950B104F1100000F095FA28B1AC
:10254000C9F80080BFF34F8FBFF36F8FFFF77AFD9D
:10255000012006B0BDE8F087059808B126B107E074
:10256000FFF770FD0020F4E701A8FFF7C5FD012685
:10257000FFF768FDFFF754FEFFF756FD94F944009E
:10258000401C01D184F8447094F94500401C01D1ED
:1025900084F84570FFF756FD05A901A800F0C8F8BA
:1025A00058B12046FFF754FC00F0C2FA2046FFF76E
:1025B000F5FB0028B3D00020CBE72046FFF7EEFB69
:1025C00090B104F124000599FFF7A4FD2046FFF720
:1025D0003FFC00F0ADFA0028A1D1C9F80080BFF39C
:1025E0004F8FBFF36F8F9AE72046FFF731FC00F063
:1025F0009FFA94E704ED00E008B5002300930A4633
:102600006946FFF781FF009808BD00002DE9F343FC
:1026100083B004460025A94600264FF08057DFF816
:102620000C81FFF701FDA06BC8B1401EA0632068BC
:1026300010B9FFF79BFCA060206950B104F11000B5
:1026400000F012FA28B1C8F80070BFF34F8FBFF343
:102650006F8FFFF7F7FC012005B0BDE8F083049809
:1026600008B125B107E0FFF7EDFC0020F4E701A871
:10267000FFF742FD0125FFF7E5FCFFF7D1FDFFF76E
:10268000D3FC94F94400401C01D184F8446094F9CF
:102690004500401C01D184F84560FFF7D3FC04A934
:1026A00001A800F045F8C8B12046FFF7D1FB00F0C3
:1026B0003FFA2046FFF772FB0028B2D0B9F1000FB5
:1026C0000AD0FFF7B1FC2046FFF787FA0146A06861
:1026D000FFF730FDFFF7B6FC0020BDE72046FFF70F
:1026E0005DFBE0B1206838B9FFF79EFCA06800F000
:1026F00061F98146FFF7A6FC04F124000499FFF775
:1027000009FD2046FFF7A4FB00F012FA002888D14B
:10271000C8F80070BFF34F8FBFF36F8F81E720467B
:10272000FFF796FB00F004FA7BE7000004ED00E001
:102730002DE9F04106460D46FFF776FC1148C368C7
:1027400074681A1B29684F1C0AD03768D0F820C05B
:102750000020674506D09C4204D8012428600CE084
:1027600000240AE0914206D9881A28603046FFF713
:10277000C3FC002401E028600124FFF763FC20462D
:10278000BDE8F0811C0000202DE9FF5F8146DDE9F6
:102790000E788A4616469B46B000FFF797FB054623
:1027A00028000ED05420FFF791FB04462CB1542191
:1027B0002046FDF752FD256304E02846FFF74EFC56
:1027C00000E000248CB10020CDE90240CDE9007882
:1027D0005B46324651464846FFF752FA2046FFF71D
:1027E00035F9012004B0BDE8F09F4FF0FF30F9E764
:1027F00005484169002903D0406B18B1002070479B
:1028000001207047022070471C0000202DE9F04194
:102810000025434E706B002805D0B069401CB061A4
:102820002846BDE8F081F468641CF46044B9B06BDC
:10283000F16BB163F063306A401C3062FFF7F0FA6D
:10284000B06A384F84420FD34FF0000CB06B006871
:1028500038B1B06BC068C1684868844212D2B062B7
:1028600002E04FF0FF30B0623068C06A00EB8000D9
:1028700057F82000012800D90125F0690028CFD0A1
:102880000125CDE74A69D1E902309860D1E9020318
:10289000586050680B1D984201D1C8685060C1F85B
:1028A00014C01068401E10608A6A9AB1D1E907808E
:1028B000C8F80800D1E90708C8F80400506801F119
:1028C0001808404501D1086A5060C1F828C0106856
:1028D000401E1060C86A0122D6F81080824042EA89
:1028E0000802326100EB800007EB800042688A60DA
:1028F0009068C860906843609360C86A00EB80008D
:1029000007EB80024A6157F82020521C47F820202C
:10291000C86A3168C96A884298D9012596E70000DB
:102920001C0000200C01002010B504460020002CE3
:102930003BD0A16C491EA164636CE26A9A4234D018
:10294000002932D1201DFFF72FFB1849012230B991
:1029500094F82C000B6902FA00F083430B61606C61
:10296000E062C0F10400A061E06A0B6982401A4392
:102970000A610F4A00EB800002EB80004068A06013
:102980008168E1608368211D59608160E06A00EB25
:10299000800002EB80006061E06A00EB800052F88A
:1029A0002010491C42F82010012010BD1C000020FE
:1029B0000C01002070B504460020002C48D0284DA2
:1029C000E16A2A68D26A914243D2A069002804DBF6
:1029D0002868C06AC0F10400A061E06A214E00EBE3
:1029E0008000616906EB800081422DD1201DFFF738
:1029F000DBFA012130B994F82C002A6901FA00F0C1
:102A000082432A612868C06AE0622A6981401143D2
:102A1000296100EB800006EB80004068A0608168BF
:102A2000E1608268211D51608160E06A00EB8000F6
:102A300006EB80006061E06A00EB800056F8201031
:102A4000491C46F8201002E02868C06AE0620120B4
:102A500070BD616C2A68D26A9142F9D2012070BDC2
:102A60001C0000200C01002070B5C068C068816A9D
:102A7000D0E907329A60D0E907235A604B6800F129
:102A80001802934201D1036A4B60002585620B68EE
:102A90005B1E0B60244B596B012499B1234D69686F
:102AA000C1618E6806628E6872608A60856229687C
:102AB000491C2960C06A1968C96A884232D9012054
:102AC000DC6170BD4169D0E90262B260D0E90226E2
:102AD00072604E68021D964201D1C6684E60456123
:102AE0000D686D1E0D60C16A1E6904FA01F535435B
:102AF0001D610E4D01EB8101783D05EB81014968B7
:102B000081608E68C6608E6872608A60C16A01EBFF
:102B1000810105EB8102426155F82120521C45F8E4
:102B20002120C7E7002070BD1C0000208401002088
:102B30002DE9F0410024A046FFF776FA3E4D686B80
:102B4000401E6863686B002871D1A86800286ED0A9
:102B500000273A4A01264EE0D068C468A16AD4E949
:102B600007309860D4E9070358604B6804F11800F7
:102B7000834201D1206A4860A7620868401E08604D
:102B80006169D4E902309860D4E9020358604B6867
:102B9000201D834201D1E3684B6067610B685B1EB7
:102BA0000B60E16AD5F810C006FA01F343EA0C03A2
:102BB0002B61224B01EB8101783B03EB81014968DA
:102BC000A160D1F808C0C4F80CC0D1F808C0CCF896
:102BD00004008860E06A00EB800003EB8001616123
:102BE00053F82010491C43F82010E06A2968C96A8C
:102BF000884200D3EE6110680028ADD10CB1FFF718
:102C00000FF9AC693CB1FFF701FE00B1EE61641E43
:102C1000002CF8D1AF61E86948B14FF001080849CC
:102C20004FF080500860BFF34F8FBFF36F8FFFF7F7
:102C300009FA4046BDE8F0811C0000208401002014
:102C400004ED00E0000000000000000001020304A9
:102C5000060708091051FF1F1451FF1F1851FF1FCD
:102C60004851FF1F4C51FF1F0056FF1F0456FF1F06
:102C70000052FF1F0452FF1F4051FF1F4451FF1F0E
:102C80000852FF1F2051FF1F2451FF1F2851FF1F13
:102C90002C51FF1F3051FF1F3451FF1F08220240EB
:102CA0000C2202402022024028220240242202401C
:102CB0001C2202402C220240102202401422024018
:102CC00018220240FF0FFF0FFF0000000F001F003F
:102CD000FF07FF1FFF07FF073F003F003F00000007
:102CE000FFFFFFFFFFFFFFFFFF0FFF0F00000000D0
:102CF00001020304142D00080000002080000000E1
:102D0000DC170008942D000880000020402D0000F2
:102D1000EC17000800127A0000000000000000001C
:102D2000000000000100000008000000000000009A
:102D30000000000000000000000000000000000093
:102D40000000000000000000000000000000000083
:102D50000000000000000000000000000000000073
:102D60000300000000000000000000000000000060
:102D70000000000000000000000000000000000053
:102D8000000000000000000000000000AAAAAAAA9B
:042D9000000000003F
:0400000508000131BD
:00000001FF
